:020000040000FA
:100000008B018A018301CA28F000030E8301F100ED
:100010000408F2008C1E4C28981C18194928181C3A
:1000200028283711B6011A08B100B7196328603AB9
:10003000031925283108320603194128A03A03196B
:100040002528603A03193C286328B5013715632831
:100050002030360784001A08371D63288000B50653
:10006000B60A20080F39023E3606031D63283711F1
:10007000B5080319B71563280614203099009900B4
:100080005A28371C6328061483160C168312B714DB
:1000900050281A08181218160C1E6328B71C5A2864
:1000A000A0303307840000089900B30AB40B63281A
:1000B0003710B7108316981C5B280C128312602827
:1000C00061286228061072088400710E8300F00E09
:1000D000700E090082073F3406345B344F346634B7
:1000E0006D347D3407347F346F343F0E0739820717
:1000F0000134023404340834103420344034803461
:1001000000348207013402340434083410342034BB
:100110004034003480348207013400340034003429
:1001200000348034403408341034820700341034F2
:100130002034403480340034003400340034BD199D
:10014000CF01CF08031908000301CF1A01304F1B5C
:100150000230CF180330CF01510782070F2B572BE6
:10016000242B6A2B2D2B162B1F2B6A2B5B2B392B49
:100170005F2B6A2B0800842B902BCA28842B6F2BB3
:100180007C2BCA28842B9E2B992BCA283D2B292BEC
:10019000272B6A2B9801850186018316F63086008D
:1001A000FF30850020308C00813081000B308E00C4
:1001B00000309F00831205309F00203084008001B2
:1001C000840A841FDF28C92264224524C323C03047
:1001D0008B004030C900CA0075224D184C290130EF
:1001E0005824BF006030C1000C22092141210C18A5
:1001F00046213718F628112209215B23FD222322EC
:100200003C1641210C1C01290F214121CE239F20A6
:100210000529313090008E018F010C1008009001EB
:100220000C1008000C1C1B290F21D108031D1B29D1
:100230003F08D522EB228C1C08008C109F1F25291B
:10024000C7304306031DC30A2829C308031DC3037F
:10025000430C8400040C3F399500430E30390C38B0
:1002600097004308C5070318C60AC40F08004608CC
:10027000C800C501C6013C170310CC0D03184C146F
:10028000080012217B22B719522108000C10F93006
:10029000C9000730CA0008008623342412217B22BB
:1002A0009F204D292008613A031D82292108031D42
:1002B0006429BD180A2ABD11BD143D10F930C900CA
:1002C0003F30CA00EB22082A013A031D7429BD11F0
:1002D000BD103D103F08D522EB223D080B39031914
:1002E000082AB7112322082A033A031D0A2ABD1936
:1002F0000A2ABD15BD103D106D30C9007330CA000B
:10030000EB22082A033A031D92292108223A031DF1
:100310000A2A2208BD00BD197C29BD185E293D1896
:10032000AA296A29013A031D9E292108213A031DA1
:100330000A2A2208B8002308B9000A2A2008813AAC
:10034000031DB0292108031D0A2A3D180A2ABD11E0
:10035000BD103D14F930C9006D30CA00EB22082AE7
:100360002008E13A031DBF292108883A031D0A2A03
:100370006D30C9004030CA00CC30CC000A2A033AA4
:10038000031DCC292108F039203A031D0A2A3C1507
:100390003F08BE00C101EC29013A031DDF292108F5
:1003A000403A031D0A2A22083F39031D0A2A23085E
:1003B0003F06031D0A2A3C14EB223C160A2A073A80
:1003C000031DFC292108F039031D0A2A3C113F08AE
:1003D000BE0023081F39C100A21BC116211CA11891
:1003E00041172119C11722087F39C0003C10A119FB
:1003F0003C14EB223C160A2A013A031D0A2A210862
:10040000F039103A031D0A2A3C152508BE00E929D7
:10041000D101EB22B711080021304F2221305722A1
:10042000602A21304F2224305722602A80304F2208
:10043000602A21304F2280305722602A21304F22FB
:1004400081305722602AE3304F220030572200309B
:1004500057223F085722602AE4304F221030411BB8
:100460001230C11B13305722003057223F08572249
:100470004008C11A803857223C10EB223F08F30095
:1004800001306124602AE4304F22203057220030AE
:1004900057223F08572241081F3957223C2ABA00E9
:1004A000B71952213718502AB301B4013A08BB00DA
:1004B000A030340784003B088000B306B40A08006B
:1004C0003308572237140800003058241F39031905
:1004D00001304038B2008400040E8406040C840607
:1004E0000419840A0418B2170800851A08004B087A
:1004F0007720CD0408000B1D08000B117522831610
:10050000D9308504F03086048312C922CC1B080040
:10051000F401F5014B0877204A050319912A0830A8
:10052000AF224B08812049050319982A0730AF22D2
:10053000BD22CB08031D08004E094D05CF0003194D
:10054000A32A3730D0004D08CE00CD014E08031944
:100550000800D00B0800CF001630D0000800F300D0
:100560008B20F40473089520F504080083167409A1
:1005700085057509860583120800B622740885046E
:10058000750886040800B622740985057509860574
:100590000800CB0A09304B060319CB014B088B200E
:1005A000F4004B089520F500C32ACA0064304A02C3
:1005B0000318E72AC9010A30C90ACA020318DC2A4B
:1005C0004A076A20CA0049036A20C9000800383077
:1005D000CA005C30E52A0301D108031D01303C1834
:1005E000CC30BD18C3303D18C330BD19C330CC006A
:1005F00008003F080F39043E0800BC12F9225824B5
:10060000F30075207305031DBC160800F922582459
:10061000F3007520F304BC1EF3065E246334383007
:10062000C900CA010430D100EB22080006233F06AE
:100630000319BF01BF0AFD2223223F08D52A062342
:10064000BF030319BF001B2B1030C106432A023021
:100650002B2B01302B2BC10643220830C11801304F
:10066000CA00083041180130C9001830D100EB220F
:1006700008002030C106BC062C22C208031D5B2BDB
:10068000C11E4B2B5E30C9000830411B4030C11BDE
:100690000130CA00532B0830411B4030C11B0130D0
:1006A000C9005E30CA000830D100EB2208002030BB
:1006B000C106BC062C22D101EB223F08D52AC20874
:1006C000031D08008030C11F4030411BC030C106EF
:1006D0002C223D2B3D181E2ABD186B2B192A0030E9
:1006E0005824F300F30A2030730601300319F30095
:1006F000003061247308D52A00305824F300F30336
:100700001F300319F300782BBC1D892BBC117730E7
:100710008B2BBC157330C900CA010C30D100080006
:100720001430BC1D1030D100BC1908000030582412
:10073000D52A4808C700F3000230612C831612083E
:100740008312F500F40108308400AB2B0310F40D84
:10075000F50D0318AF2B48087502031CB22B48088F
:10076000F5027414840BA62B7408B923F30003302C
:10077000612C8400841F041B3130841E31308316A9
:1007800092008312080003305824B9233C309200B1
:100790000C30970002305824C70008003C1F0800A6
:1007A0003C1337180800B71247080319E32B480217
:1007B0000318DC2B003CB716FC3E031C030184002D
:1007C0000310840DE52B480884003C1A222C411BA1
:1007D000F92BC11B092C0310840C0310840C03108B
:1007E000840C0E302424031908002A24031D013E22
:1007F000182C0310840C0310840C1C3024240319BF
:1008000008002A24031D033E8400040C031810383A
:10081000182C7E30242403190800C2060310420C51
:100820002C24031D013ED108031D182C4218CA17A1
:10083000C000C20803192C2A3C083706410620399B
:10084000C1062C2A3C120800040203188402040882
:10085000420608000408C200D108031D322CD5222C
:10086000CC010921420808003C1F08003C13510834
:10087000143A031D08000310480CD5224818CA1763
:10088000480847060319C91708000610B701B60142
:10089000831603309900643098008312D03098009A
:1008A0000301FF3E031D512C1A081A081A080800FC
:1008B00083169B001C141A088312080083165A24FE
:1008C000622C5824730603190800730883169A00D3
:1008D0001C158B1355309D00AA309D009C148B175E
:0A08E0001C119C18712C83120800F3
:02400E00503F21
:104200000100030000003100000000000000000079
:10421000000000000000000000000000000000009E
:104220000000000000000000530069006D007000F5
:104230006C00650020004D006100750073002000D7
:1042400076002E0034000A0046002E004300610074
:10425000C300B1006100640061002D003E004A000F
:104260002E0046007500C4008D0069006B002D0013
:104270003E0048002E0048006100660074006D009A
:1042800061006E006E000A00310039002F0030001E
:0842900032002F003000350060
:00000001FF
